S02B00002F686F6D652F766F6F72627572672F446576656C6F706D656E742F4F70656E424C542F5461726765E0
S31508000000003000207D180008CD180008CD1800081B
S31508000010CD180008CD180008CD180008000000000B
S31508000020000000000000000000000000CD180008D5
S31508000030CD18000800000000CD180008CD180008EB
S31508000040CD180008CD180008CD180008CD180008EE
S31508000050CD180008CD180008CD180008CD180008DE
S31508000060CD180008CD180008CD180008CD180008CE
S31508000070CD180008CD180008CD180008CD180008BE
S31508000080CD180008CD180008CD180008CD180008AE
S31508000090CD180008CD180008CD180008CD1800089E
S315080000A0CD180008CD180008CD180008CD1800088E
S315080000B0CD180008CD18000800000000CD1800086B
S315080000C0CD1800080000000000000000CD18000848
S315080000D000000000CD180008CD180008CD1800084B
S315080000E0CD180008CD180008000000000000000028
S315080000F000000000000000000000000000000000F2
S3150800010000000000000000000000000000000000E1
S315080001100000000000000000CD180008CD180008F7
S3150800012000000000000000000000000000000000C1
S3150800013000000000000000000000000000000000B1
S31508000140CD180008CD1800080000000000000000C7
S315080001500000000000000000000000000000000091
S315080001600000000000000000000000000000000081
S315080001700000000000000000000000000000000071
S30D0800018000000000CD1800087C
S3150800018810B5054C237833B9044B13B10448AFF3BB
S3150800019800800123237010BD3400002000000000F1
S315080001A81819000808B5034B1BB103490348AFF3F0
S315080001B8008008BD00000000380000201819000853
S315080001C872B6704762B67047F0B5002401E001348C
S315080001D8E4B2112C20D8114D15F814E005EB4405A6
S315080001E86F780EEB070606FB00064FF4FA4595FBF3
S315080001F8F6F506FB05F5B5F5FA4FE8D195FBF6F6DB
S31508000208B6B20E80013EB6B2B6F5806FDFD282F876
S3150800021800E01F700120F0BD0020F0BD5819000845
S3150800022800B583B001AB0DF105020DF106014FF4D7
S31508000238FA70FFF7C9FF012803D0E221384800F011
S31508000248BFFB384B00225A611A6842F400421A600A
S3150800025801E000F071FC334B1B6813F4004FF8D12A
S31508000268304B1A6822F002021A601A6842F0010234
S315080002781A6001E000F060FC2A4B5B6813F0010F76
S31508000288F8D09DF805305A1E9DF80430013B1B0529
S3150800029843EA0243BDF80620013A1343214AD361CB
S315080002A8136823F00103136001E000F045FC1D4BB9
S315080002B85B6813F0010FF8D11A4BD3F8002242F005
S315080002C80102C3F80022D3F81C2222F00102C3F85F
S315080002D81C22D3F80C2242F00102C3F80C22002291
S315080002E8C3F84022C3F84422D3F8042222F00102B4
S315080002F8C3F80422D3F8142222F00102C3F8142200
S31508000308D3F81C2242F00102C3F81C22D3F80022B3
S3150800031822F00102C3F8002203B05DF804FB00BF0F
S31508000328301900080064004038B504460D46214BCC
S315080003389B6813F0806F2FD01E4BD3F8802102F0EC
S315080003480102C3F88021D3F8802142F07C4242F4A6
S315080003580012C3F88021C3F88451E178A278120400
S3150800036842EA0162617842EA012221780A43C3F81F
S315080003788821E179A279120442EA0162617942EA9E
S31508000388012221790A43C3F88C21D3F8802142F047
S315080003980102C3F8802107E040F22111064800F05F
S315080003A80FFBC9E700F0C8FB024B9B6813F0806F88
S315080003B8F8D038BD00640040301900081B4BDB68CC
S315080003C813F0030F2FD0194BD3F8B02140F2676307
S315080003D8B3EB525F06D00020144AD36843F02003D3
S315080003E8D3607047114BD3F8B8210270D3F8B821F7
S315080003F8120A4270D3F8B821120C8270D3F8B821C1
S31508000408120EC270D3F8BC210271D3F8BC21120AA5
S315080004184271D3F8BC21120C8271D3F8BC311B0E79
S31508000428C3710120D8E70020704700BF0064004068
S3150800043808B5FFF7C5FE08BD10B500F0C1F900B943
S3150800044810BD00F077FD0028FAD000F02FFB00F069
S31508000458CBF900F0B9F920F0604020F07F00044B92
S31508000468186000F0B1F94468FFF7ACFEA047E7E763
S3150800047808ED00E070B508E0461C4D1C0B780370C3
S3150800048800F05AFB304629462246531E9CB2002ADB
S31508000498F2D170BD08B5C1F3080353B90368994288
S315080004A809D040F8041B4FF40072FFF7E3FF012058
S315080004B808BD002008BD012008BD2DE9F041074602
S315080004C800F086FD342000F09BFD00F09FFD012812
S315080004D816D000247F2C15D83E68A30006EB03081F
S315080004E83B445D6800F028FB2946404600F0D6FDE7
S315080004F8042809D156F824309D420BD10134E9E77E
S31508000508002402E0012400E0002400F071FD2046E2
S31508000518BDE8F0810024F8E738B50D460B4B98423C
S3150800052808D004460A4B994206D0FFF7C6FF20B9F9
S31508000538002407E0074C00E0044C29462046FFF74C
S31508000548A9FF08B1204638BD0024FBE7540200205D
S3150800055800200008500000202DE9F04106460C4608
S3150800056817461D4621F4FF7828F001080368B3F1F9
S31508000578FF3F0DD03368984505D041463046FFF70A
S31508000588CBFF064628B33368E41A344404340CE02F
S315080005984146FFF77FFF03460028EBD116E017F818
S315080005A8013B04F8013B013D0FD000F0C5FA331DA5
S315080005B8E31AB3F5007FF2D308F500713046FFF762
S315080005C8ABFF064638B1041DE9E701231846BDE81E
S315080005D8F0810023FAE70023F8E700004FF0FF331D
S315080005E8024A1360024A1360704700BF5000002091
S315080005F8540200200E4B984216D910B54318013BF1
S315080006080C4CA34212D80B46014620F4FF7020F082
S315080006180100094CA04203D00848FFF79DFF10BD0A
S315080006280748FFF799FF10BD00207047002010BD46
S31508000638FF1F0008FFFF00080020000850000020E0
S315080006485402002070B520F4FF6525F007051A4BFB
S315080006589D422CD94318013B184A93422AD8401B75
S315080006680144C1F3CF26C1F30A0109B10136B6B26E
S3150800067800F0AEFC342000F0C3FC00F0C7FC0128EB
S315080006880DD00024A6420CD900F056FA05EBC42072
S3150800069800F0E6FC042808D10134A4B2F2E70024E5
S315080006A800E0012400F0A4FC02E00024FAE7002494
S315080006B8204670BD0024FBE7FF1F0008FFFF00085F
S315080006C8104B1B68B3F1FF3F1AD000B583B00D4A2B
S315080006D8536891680B44D1680B4411690B445169F6
S315080006E80B4491690B44D26913445B4202AA42F847
S315080006F8043D04210448FFF77DFF03B05DF804FBB9
S315080007080120704754020020882100080D4B1B68F9
S315080007180D4A126813440D4A126813440C4A1268A3
S3150800072813440C4A126813440B4A126813440B4ABA
S31508000738126813440A4A1268D34201D00020704747
S315080007480120704700200008042000080820000837
S315080007580C2000081020000814200008182000089B
S315080007688821000808B50C4B1B68B3F1FF3F04D075
S315080007780948FFF7A2FE034650B1084B1B68B3F1B8
S31508000788FF3F07D00548FFF798FE034600B1012347
S31508000798184608BD0123FBE7540200205000002034
S315080007A8004870470020000808B5FFF717FF08BD7E
S315080007B808B5FFF71FFF08BD08B5FFF743FF08BDD3
S315080007C808B5FFF7A3FF08BD08B5FFF7E9FF08BD99
S315080007D808B5FFF775FF034608B9184608BDFFF7B9
S315080007E8C1FF0346F9E700000022014B1A6070476B
S315080007F810E000E008B5FFF7F7FF054B4FF6FF12C4
S315080008085A6000229A6005211960024B1A6008BDD1
S3150800081810E000E058040020044B1B6813F4803FDE
S3150800082803D0034A136801331360704710E000E0E9
S315080008385804002008B5FFF7EFFF014B186808BDF4
S315080008485804002010B504468021094800F00DFF19
S3150800085808B9002010BD2146054800F0FEFE802193
S31508000868034800F002FF0028F9D0012010BD00BF98
S315080008780044004010B504462021064800F0F5FE5D
S31508000888012801D0002010BD024800F0EAFE2070B9
S31508000898012010BD0044004010B586B04FF46143EE
S315080008A80093002301930293039305930C2304935F
S315080008B8054C6946204600F061FE0121204600F0F5
S315080008C8C1FE06B010BD00BF0044004070B506461C
S315080008D80D4640290AD82846FFF7B4FF012803D051
S315080008E879210E4800F06CF8002406E075210B48BB
S315080008F800F066F8EFE70134A4B2ABB29C420BD21B
S3150800090800F01AF9305DFFF79DFF0128F3D0822120
S31508000918024800F055F8EEE770BD00BF7C190008DC
S3150800092838B5224B1C78ACB92148FFF7A3FF012834
S3150800093801D0204638BD1E4B1B78002BF9D0FFF78F
S3150800094879FF1C4B186000221B4B1A700122174BA3
S315080009581A70EEE70546184B1B78013314481844F5
S31508000968FFF788FF044601280AD0FFF763FF114BF3
S315080009781B686433984216D900240C4B1C70D8E7B8
S315080009880D4B1A780132D2B21A70094B1B789A4263
S3150800099801D00024CDE709492846FFF76BFD002258
S315080009A8024B1A70C5E70024C3E700BF9D04002060
S315080009B85C040020A00400209E0400205D0400209A
S315080009C808B500F0B9F8FCE708B500F0ADF8012855
S315080009D803D0094B1B78012B00D008BDFFF72AFF67
S315080009E8064B1B6803F5FA739842F6D30022024BA6
S315080009F81A70FFF721FDF0E7A4040020A8040020D8
S31508000A0808B50122044B1A70FFF714FF034B186048
S31508000A18FFF7DAFF08BD00BFA4040020A8040020D9
S31508000A2808B5FFF705FD00F083F8FFF7E3FEFFF7C3
S31508000A38BBFE00F00DF8FFF7E3FF08BD08B500F0A8
S31508000A487BF8FFF7E9FE00F013F8FFF7BDFF08BDCE
S31508000A5810B500F0DDF9FFF7E3FB044C012323701A
S31508000A68FFF71AFF0023237010BD00BF00000020FF
S31508000A7808B50C48FFF7A2FC012805D00948FFF776
S31508000A884FFF012807D008BD0122074B1A700548F1
S31508000A9800F0DEF9F2E70022034B1A70014800F06D
S31508000AA8D7F9F0E7AC0400200000002070470000E2
S31508000AB838B504460D46094B1B78012B05D0074B5C
S31508000AC81B7833B100F0BCF938BDC9B2FFF72CFC66
S31508000AD8F5E7E9B22046FFF7F9FEF3E7000000203C
S31508000AE8074B1B78022B05D0032B05D0012B05D005
S31508000AF8402070470020704700207047082070473C
S31508000B0800000020074B1B78022B05D0032B05D0C5
S31508000B18012B05D0402070470020704700207047F9
S31508000B28082070470000002008B500F07FF908BDC6
S31508000B3808B500F00BFA08BD08B500F00CFA08BDB0
S31508000B4810B4002304E010F8011B0B44DBB221465D
S31508000B584C1E0029F7D1136001205DF8044B704735
S31508000B680022014B5A707047EC040020034BFE2202
S31508000B78DA7018710222A3F844207047EC040020A2
S31508000B8810B5054C00232370FFF7EAFFFF23E3702F
S31508000B980123A4F8443010BDEC040020064BFF22BC
S31508000BA8DA7000221A71597859719A71DA711A72BB
S31508000BB80622A3F844207047EC04002008B5002054
S31508000BC8FFF7D4FF08BD0000074BFF22DA70074A73
S31508000BD89A6400221A715A719A710722C3F8072073
S31508000BE80822A3F844207047EC040020A819000836
S31508000BF8044BFF22DA7042689A640122A3F844205B
S31508000C08704700BFEC04002010B5084CFF23E370BA
S31508000C18E21D4168A06CFFF793FF207100236371FA
S31508000C28A3710823A4F8443010BD00BFEC040020C3
S31508000C3808B53120FFF79AFF08BD000038B5084CFB
S31508000C48FF23E370002525716571FFF749FFA07139
S31508000C58E571257265720723A4F8443038BD00BFCC
S31508000C68EC04002038B5FFF77BFF0E4C01252570EC
S31508000C78FF23E3701023237100236371FFF730FF06
S31508000C88A071FFF73FFFE071FFF73CFFC0F30720AD
S31508000C9820726572A5720823A4F84430FFF784FD0C
S31508000CA838BD00BFEC04002038B505464478FFF780
S31508000CB817FF0138844210DC0A4C6A78A16C201D9B
S31508000CC8FFF7D8FBFF23E3706A78A36C1344A36481
S31508000CD86B780133A4F8443038BD2220FFF746FF65
S31508000CE838BD00BFEC04002038B504464578FFF740
S31508000CF8F7FE0138854211DC61680A4DA9646278F5
S31508000D08281DFFF7B7FBFF23EB706278AB6C13441B
S31508000D18AB6463780133A5F8443038BD2220FFF761
S31508000D2825FF38BDEC04002038B505460D4B9C6CEC
S31508000D38FFF7D6FE6A1C411E2046FFF739FD60B14B
S31508000D48084CFF23E370FFF7CBFE0138A36C034476
S31508000D58A3640123A4F8443038BD3120FFF706FF01
S31508000D6838BD00BFEC04002038B504464578FFF7BF
S31508000D78B7FE023885420EDC114BFF22DA700122D3
S31508000D88A3F84420617851B9FFF722FD90B93120BC
S31508000D98FFF7ECFE38BD2220FFF7E8FE38BDA21C97
S31508000DA8074B986CFFF704FD28B16178044A936CE1
S31508000DB80B44936438BD3120FFF7D8FE38BD00BF11
S31508000DC8EC04002008B54168074B986CFFF7F4FC5B
S31508000DD830B1054BFF22DA700122A3F8442008BD7A
S31508000DE83120FFF7C3FE08BDEC04002008B5FFF75D
S31508000DF823FB034BFF22DA700122A3F8442008BD1F
S31508000E08EC04002008B589B2FFF752FE08BD0000B9
S31508000E18054B00221A709A6483F84320A3F84420E5
S31508000E289A705A70704700BFEC040020034B1B7871
S31508000E380BB1012070470020704700BFEC04002062
S31508000E480022024B83F84320704700BFEC040020B9
S31508000E5808B50378FF2B04D0354A1278012A14D02E
S31508000E6808BDFFF7FFFE324B93F84330012B5AD0E3
S31508000E782F4BB3F944100029F2DD1846012380F8F0
S31508000E8843300330FFF7BEFFEAE7C93B352B46D8A0
S31508000E98DFE803F03345454245453F363C39454585
S31508000EA845454545454545454545454545454545DC
S31508000EB84545454545454545454545454545241E14
S31508000EC81B2145454527452A2D30FFF7EDFECAE77C
S31508000ED8FFF70AFFC7E7FFF78BFEC4E7FFF794FE9D
S31508000EE8C1E7FFF771FEBEE7FFF768FEBBE7FFF746
S31508000EF855FEB8E7FFF744FEB5E7FFF715FFB2E773
S31508000F08FFF732FFAFE7FFF799FEACE7FFF75AFF9F
S31508000F18A9E7FFF76BFFA6E7FFF78AFEA3E72020F6
S31508000F28FFF724FE9FE71020FFF720FEA0E700BF83
S31508000F38EC04002008B500F043F84FF400714FF0B0
S31508000F48904000F025F900B1012008BD08B56420D5
S31508000F5800F006F808BD08B500F008F808BD000056
S31508000F68014B1880704700BF3805002008B5FFF701
S31508000F7861FC0F4B1B68984210D30E4B1B7873B94C
S31508000F8801220C4B1A7008210B4800F008F9FFF7E4
S31508000F9851FC0A4B1B881844054B186008BD0022EB
S31508000FA8044B1A700821044800F0FBF8EFE700BF65
S31508000FB83C0500203A0500200004004838050020B2
S31508000FC808B50821014800F0ECF808BD00040048F7
S31508000FD8054B1B6913F0800F05D0034B034A5A606B
S31508000FE802F188325A60704700200240230167459B
S31508000FF8024A136943F080031361704700200240D0
S31508001008014BD860704700BF002002400B4BDB68D5
S3150800101813F0010F0DD1094BDB6813F0100F01D03F
S3150800102802207047054BDB6813F0040F03D0032032
S315080010387047012070470420704700BF002002400F
S3150800104810B50446FFF7E2FF02E0FFF7DFFF013CB1
S31508001058012801D1002CF8D104B9052010BD0000DB
S3150800106838B505464FF43020FFF7EAFF042800D0C4
S3150800107838BD094C236943F0020323616561236976
S3150800108843F0400323614FF43020FFF7D9FF236963
S3150800109823F002032361EBE70020024030B583B052
S315080010A805460C46002301934FF43020FFF7C8FF86
S315080010B8042801D003B030BD104A136943F0010370
S315080010C81361A3B22B804FF43020FFF7B9FF042829
S315080010D805D00A4A136923F001031361EAE70235C2
S315080010E80195019B240C1C804FF43020FFF7A8FFBC
S315080010F8024A136923F001031361DBE70020024063
S3150800110800230F2B43D8F0B434E085685F00032624
S31508001118BE4025EA0605856082684C79BC402243AC
S3150800112882608588ADB29FB20126BE4025EA0605CB
S315080011388580828892B28C79BC40A4B22243828088
S3150800114802685D00032404FA05F622EA060202602C
S3150800115802680E79AE4032430260C2689EB27600D3
S31508001168B44022EA0402CC79AC402243C260013377
S315080011780F2B0AD801229A400C68A243F7D10A799C
S31508001188013AD2B2012ADBD8BFE7F0BC70477047EC
S31508001198038A194201D100207047012070478161EE
S315080011A870470185704730B401F007039B009A40E1
S315080011B8C908083150F821400F2505FA03F324EA2F
S315080011C8030340F8213050F821301A4340F821200B
S315080011D830BC7047F0B5A04B5A6802F00C02042AD6
S315080011E83AD0082A3CD01AB19C4B0360002201E089
S315080011F89A4B0360984D6B68C3F30313DFF864E2F0
S315080012081EF80370FFB2016821FA07F343606C6899
S31508001218C4F302241EF80440E4B223FA04F48460F2
S315080012286E68C6F3C2261EF80660F6B2F340C360B7
S31508001238ED6A2D0905F00F0CDFF82CE23EF81CE0E4
S315080012481FFA8EFE15F0100F23D0BEF1000F20D01E
S31508001258B2FBFEF505611DE0804B03600022C9E775
S315080012687D4B5A685B68C2F38342023213F4803FA7
S3150800127804D17B4B03FB02F20260BBE7764BDB6AC1
S3150800128803F00F0301337549B1FBF3F303FB02F2CD
S31508001298F2E70161704DED6A6D0A05F00F0CDFF88B
S315080012A8C8E13EF81CE01FFA8EFE15F0100F06D0AE
S315080012B8BEF1000F03D0B2FBFEF5456100E04161BF
S315080012C8654D2D6B15F0100F40F08180634D8561D3
S315080012D8614D2D6B15F0200F7BD1604DC5615E4DB4
S315080012E82D6B15F0400F76D15C4D05625A4D2D6B66
S315080012F815F4807F01D08A426FD04362564D2D6B14
S3150800130815F4805F01D08A426CD08362524D2D6BEA
S3150800131815F4007F01D08A4269D0C3624E4D2D6B01
S3150800132815F4806F01D08A4266D0C3644A4D2D6B86
S3150800133815F4006F01D08A4263D00365464D2D6BBC
S3150800134815F4005F01D08A4260D00365424D2D6BC3
S3150800135815F4004F01D08A425DD083653E4B1B6B5E
S3150800136813F0030F5CD184633B4B1B6B13F4403FAC
S315080013787CD1C463384B1B6B13F4402F40F095801F
S315080013880464354B1B6B13F4401F40F0AD8044646E
S31508001398314B1B6B13F4400F00F0C5802E4B1B6BAB
S315080013A803F44003B3F5800F00F0BF802A4B1B6B8C
S315080013B803F44003B3F5000F00F0B980264B1B6B06
S315080013C803F44003B3F5400F00F0B580F0BD816122
S315080013D87EE7C16183E7016288E7B7428DD1550088
S315080013E845628BE7B74290D1550085628EE7B742CA
S315080013F893D15500C56291E7B74296D15500C564A1
S3150800140894E7B74299D15500056597E7B7429CD145
S31508001418550045659AE7B7429FD1520082659DE710
S315080014280D4B1B6B03F00303012B0ED00A4B1B6BEA
S3150800143803F00303022B0AD0074B1B6B03F00303C5
S31508001448032B91D1054B83638EE781638CE74FF4B1
S315080014580043836388E700BF0010024000127A0041
S3150800146800093D002400002004000020334B1B6BB4
S3150800147803F44033B3F5803F11D0304B1B6B03F4AC
S315080014884033B3F5003F0CD02C4B1B6B03F44033A9
S31508001498B3F5403F7FF46EAF294BC3636AE7C16370
S315080014A868E74FF40043C36364E7244B1B6B03F4F4
S315080014B84023B3F5802F11D0204B1B6B03F4402330
S315080014C8B3F5002F0CD01D4B1B6B03F44023B3F563
S315080014D8402F7FF456AF1A4B036452E7016450E76E
S315080014E84FF4004303644CE7144B1B6B03F4401397
S315080014F8B3F5801F11D0114B1B6B03F44013B3F5DA
S31508001508001F0CD00D4B1B6B03F44013B3F5401F9B
S315080015187FF43EAF0A4B43643AE7416438E74FF431
S315080015280043436434E78464F0BD8164F0BD4FF436
S3150800153800438364F0BD024B836447E7001002400A
S3150800154800127A0029B9054A536923EA000050614E
S315080015587047024A536918435061704700100240A1
S3150800156829B9054AD36923EA0000D0617047024AB7
S31508001578D3691843D06170470010024030B599B056
S3150800158804460D46036823F001030360436823F401
S3150800159840538A6813434360036823F4B05323F01F
S315080015A80C034A68C9680A4329690A43134303604E
S315080015B8836823F440736A691343836001A8FFF7B5
S315080015C809FE1C4B9C4227D01B4B9C4226D01B4B22
S315080015D89C4225D01A4B9C4224D01399236813F4AD
S315080015E8004F21D049002A68B1FBF2F302FB131217
S315080015F82968B2EB510F00D30133226812F4004F61
S3150800160806D0C3F3420223F00F031B041B0C134333
S315080016189BB2A38119B030BD0F99DFE71099DDE7B2
S315080016281199DBE71299D9E72A68B1FBF2F302FBAD
S315080016381312DDE700380140004400400048004026
S31508001648004C004021B9036823F001030360704782
S31508001658036843F0010303607047C1F30801018575
S315080016687047808CC0F308007047C3690B4201D1E4
S3150800167800207047012070471222164B1A60A3F5FE
S3150800168880535A685A605A685A605A6842F480629F
S315080016985A605A6822F47C125A605A6842F46012F0
S315080016A85A601A6842F080721A600B4B1B6813F06E
S315080016B8007FFAD0084B5A6822F003025A605A6823
S315080016C842F002025A60044B5B6803F00C03082BCD
S315080016D8F9D17047002002400010024010B5174C97
S315080016E8D4F8883043F47003C4F88830144B1A6861
S315080016F842F001021A605968124A0A405A601A6882
S3150800170822F0847222F480321A601A6822F480223F
S315080017181A605A6822F4FE025A60DA6A22F00F0240
S31508001728DA62196B084A0A401A6300229A60FFF7B8
S31508001738A3FF4FF00063A36010BD00BF00ED00E0F3
S31508001748001002400CC07FF8CCFC00FF2DE9F041E0
S3150800175882B001214FF48020FFF7F4FE4FF0080805
S31508001768CDF8008001248DF8044000258DF8065030
S3150800177803268DF805608DF80750394F69463846AF
S31508001788FFF7BEFC41463846FFF70BFD21464FF4E6
S315080017980030FFF7D7FE8DF804508DF807404FF450
S315080017A80073009369464FF09040FFF7A9FC21465D
S315080017B84FF40030FFF7D4FE21464FF40030FFF708
S315080017C8C1FE072202214FF09040FFF7ECFC0722E2
S315080017D80F214FF09040FFF7E6FC8DF806508DF87C
S315080017E8074002278DF80470042300938DF80560D6
S315080017F869464FF09040FFF783FC8DF804704FF464
S315080018080043009369464FF09040FFF779FC21465C
S315080018184FF40030FFF796FE09220B214FF090404F
S31508001828FFF7C1FC09220C214FF09040FFF7BBFCDB
S315080018384FF4C05300938DF804708DF805608DF841
S3150800184806508DF8074069464FF09040FFF758FC58
S3150800185821464FF00070FFF783FE02B0BDE8F0811D
S315080018680004004808B5FFF771FFFFF7D9F8FFF736
S31508001878E5F8FCE7DFF834D0002103E00C4B5B58A9
S31508001888435004310B480C4B42189A42F6D30B4A7C
S3150800189802E0002342F8043B094B9A42F9D3FFF7C2
S315080018A81DFF00F011F8FFF7DDFFFEE70030002006
S315080018B8B819000800000020340000203400002071
S315080018C840050020FEE7000070B50D4E0D4CA41B20
S315080018D8A4100025A54209D10B4E0C4C00F018F8A7
S315080018E8A41BA4100025A54205D170BD56F82530BD
S315080018F898470135EEE756F8253098470135F2E757
S31508001908B0190008B0190008B0190008B419000879
S31508001918F8B500BFF8BC08BC9E467047F8B500BFC6
S30D08001928F8BC08BC9E46704796
S315080019302E2E2F2E2E2F2E2E2F2E2E2F536F7572C4
S3150800194063652F41524D434D345F53544D333246F0
S31508001950332F63616E2E6300050206020603070332
S315080019600803090309040A040B040C040C050D05F5
S315080019700E050F050F061006100710082E2E2F2E1F
S315080019802E2F2E2E2F2E2E2F536F757263652F41F5
S31508001990524D434D345F53544D333246332F7561A0
S315080019A072742E63000000004F70656E424C54003E
S309080019B0AD0100086F
S309080019B4890100088F
S315080019B804000000010002000400060008000A00EE
S315080019C80C00100020004000800000010000000004
S315080019D800000000000000000102030401020304DD
S309080019E806070809CF
S7050800187D5D
